:1000000011298030A100FE30AF200130AF207530C3
:10001000A7003030C628A101A117AF00AF08031D0B
:100020001328030114280130AF020310A20CA20C04
:10003000A20CC0302205403EAF07FE30AF202F0893
:10004000AF28A101A117AF00FE30AF202F08AF28C5
:10005000A401AA00AB01A01124080319A0150530C2
:10006000A3002730A900103041200330A900E83058
:100070004120A90164304120A9010A3041202A0809
:100080004828A8002B08A7002A08A600DA2026087E
:10009000A600A3030319A011240803195228230260
:1000A000031859282608031DA011A0195928303E0D
:1000B000AF280800A300240803190C292308AF2047
:1000C000A4035B28AD000611861183160611861164
:1000D0000F30860583122D08A0188C283E30A7000B
:1000E0008030C6203330AC00A0201330A700883009
:1000F000C620A0206430C520A0206430C520223056
:10010000AC00A02028308B200C308B2006308B20B8
:10011000A0142D088C282014AC00201C9A288611CD
:10012000033C031C9F289F200530A700DC30C6201D
:10013000031408002014FE3C0319AD288615201C6A
:10014000201006150F3086052C08F039860406119C
:10015000AC0E2018A0283230C5202D080C29A11B78
:10016000622883178001840AFF3E031DB2280C29F0
:10017000A901A800FF30A807031CA907031C0C292C
:100180000330A700DF30C620BA28A701E83EA6004A
:10019000A709FC30031CCF28A6070318CC28A60704
:1001A0000000A70FCC282618D528A61CD9280000A7
:1001B000D9280800AB01AA011030AC00270DAA0D08
:1001C000AB0D2808AA022908031C290FAB0203184B
:1001D000F0282808AA0729080318290FAB070310DD
:1001E000A60DA70DAC0BDE2826080C291030B00098
:1001F000A701A601AD0CAC0C031C04292808A60716
:1002000029080318290FA707A70CA60CAB0CAA0CEA
:10021000B00BFA282A080C29831383120313000059
:100220000800A00107309F00E03083168500FF30F2
:10023000860081138312850186012030840060309E
:10024000B220A03084005030B22020308400303002
:10025000B120C830B82001207730622062206220AF
:100260002E3062207030622069306220633062205C
:100270006230622061306220733062206930622017
:10028000633062202E3062206E3062206C3062203B
:100290000B30A900B830B92001204430622043302F
:1002A00062204630622031306220363062204E308B
:1002B00062204C3062204130622020306220622077
:1002C000563062202D3062203230622001204C30C6
:1002D000622044306220523062202030622061303F
:1002E00062206630622072306220653062206730A2
:1002F0006220653062206C306220653062206E3092
:10030000622086188929851F8729051488290510E8
:1003100081290120533062206930622067306220D9
:100320006E3062206130622062206C3062202030AA
:1003300062207A3062206F306220653062206B303C
:100340006220653062206E306220361405128316FA
:10035000051283122B2AC3013C03A500C9014908D9
:100360002502031CC429E721B61CC2294308A600A4
:100370004908A200A601A20A0314A60DA20BBD29DA
:100380002608C304C90FAF29B2014308B100B20C5B
:10039000B10CB20CB10CB20CB10CB20CB10C0F30F0
:1003A000B2053208AD003108AC00A9010A30A8003E
:1003B000F620B1002B08B200B4014308B3000F309F
:1003C000B3050030B40531083307C3000800BA0193
:1003D000B9010618FC290130B820B90A0319BA0A74
:1003E0000B303A02031CFB29031DFA29B9303902EC
:1003F000031CFB29692CE9299B30B8200618B61488
:10040000061CB610361C152A440EB100B200F0309E
:10041000B1050F30B2053208A7003108A600A901C6
:100420003A30A800DA20BD001E2A03013619013E29
:10043000B618013A03193611031D3615C40A85147E
:100440000130A900F430B9208510A901F030A800CE
:100450002808B9200800BB01C4013612361ABB2A8D
:10046000BA01B901061C452AB90A0319BA0A0130B2
:10047000B820AF303A02031C442A031D432AC93076
:100480003902031C442A692C322ABA01B901061820
:10049000772AB90A0319BA0A0A30B82036186B2A23
:1004A00039080B3A3A04031D562A6A2A3908193AC0
:1004B0003A04031D5D2A85146A2A39084B3A3A0426
:1004C000031D642A85106A2A3908FA3A3A04031D82
:1004D0006A2A692C762A11303A02031C762A031DF7
:1004E000752A95303902031C762A692C472A413037
:1004F0003B02031C7C2A692CBB0A3A08031D842A90
:1005000065303902031C852A3616361CBA2A3B0E82
:10051000B100B200F030B1050F30B2053208A700CB
:100520003108A600A9014130A800DA20BD008030C2
:10053000A100803021205330622069306220673072
:1005400062206E3062206130622062206C30622056
:100550002030622067306220653062207630622071
:100560006F3062206E30622064306220653062201D
:100570006E3062202E2A361CDD2A0120493062208E
:100580006E306220693062207430622069306220EF
:10059000613062206C3062206930622073306220EA
:1005A0006530622072306220653062206E306220D9
:1005B0002E30622062206220422B0B30BD000130C1
:1005C000A2003D080B20A101B61DF52A3B304102D7
:1005D0000318EC2AC10AF42AC10117304502031896
:1005E000F32AC50AF42AC501F92A4208C1004608BF
:1005F000C500051B092B4508031D012B0C30C70046
:10060000082B0D304502031C082B0C304502C70097
:100610000D2B4508C700203062200A30470203181E
:10062000132B203062208030A100470828203A3068
:1006300062200230A40041082920051B2B2B0C301E
:1006400045020318262B61306220282B703062206F
:100650000E30BD002D2B0F30BD00410803190130B5
:10066000031D0301B5001E30410203190130031DB3
:1006700003013504B5000130861803013504031960
:10068000422B412C361E3F2CE7210130C9000F3090
:10069000490203184E2BE721C90F472B3611B6111B
:1006A000E721E721E721B61C572B0514582B05102D
:1006B0001230C900143049020318612BE721C90F19
:1006C0005A2BE7210730BC00AB214308C200E721C9
:1006D000361D6B2BB6150630BC00AB214308C60097
:1006E000E721361D742BB6150630BC00AB2143083C
:1006F000BE000330BC00AB214308C8000530BC007D
:10070000AB214308C0000830BC00AB214308BF0048
:10071000E721361D8C2BB615361C922BB619912B62
:1007200036100120B6193E2C8030A100C0302120A7
:100730001030A40020305A208030A10080302120C9
:100740003E0828202030622001304002031DAF2BDC
:100750006A306220613062206E306220272C0230C5
:100760004002031DBA2B6630622065306220623081
:100770006220272C03304002031DC52B6D30622000
:100780007230622074306220272C04304002031D36
:10079000D02B613062207030622072306220272CB2
:1007A00005304002031DDB2B6D3062206530622076
:1007B00069306220272C06304002031DE62B6A3088
:1007C0006220753062206E306220272C0730400294
:1007D000031DF12B6A306220753062206C3062207C
:1007E000272C08304002031DFC2B6130622075303D
:1007F000622067306220272C09304002031D072C3D
:10080000733062206530622070306220272C0A30FD
:100810004002031D122C6F3062206B306220743056
:100820006220272C0B304002031D1D2C6E306220ED
:100830006F30622076306220272C0C304002031D7E
:10084000272C643062206530622063306220051BF3
:10085000342C203062208030A1000230A4003F08F8
:100860002920203062203E2C203062202730622058
:100870008030A1000230A4003F082920402C692CC0
:100880002B2A851F482C05128316051283124A2C29
:100890008316051683129B30B820410803190130D6
:1008A000031D0301B5000130861803013504031947
:1008B0005A2C0515851585140130A900F430B9208E
:1008C0000511851185100130A9004A30B920C40AEC
:1008D000452B0120473062206530622062206E3057
:1008E00062202030622073306220693062206730DD
:1008F00062206E3062206130622062206C306220A3
:10090000203084006030B220A03084005030B2200B
:10091000203084003030B1200618B616061CB612FE
:1009200003010618013EB61A013C031D9D2CB70AAF
:100930000319B80A0130B820902C0301B61A01300F
:10094000013A0319B612031DB61603010618013E3B
:10095000B61A013C031DB22CB70A0319B80A0130BC
:10096000B820A52C03303802DE30031937020318F3
:06097000802C36142B2A36
:02400E00503F21
:00000001FF
